:100000000C94BB010C94CD010C94CD010C94F9011E
:100010000C94811D0C94CD010C94CD010C94CD0158
:100020000C94CD010C94CD010C94CD010C94C6160A
:100030000C94CD010C94CD010C94CD010C94CD0108
:100040000C947A160C94CD010C94C01A0C94421B9B
:100050000C94CD010C94CD010C94CD010C94CD01E8
:100060000C94CD010C94CD0138303E3041304430F9
:10007000493051305930F430F430F4306630693062
:1000800072307B30F430F430F430F430F430F4304B
:10009000873091309D30A530A830B130BA30C030B3
:1000A000F430F430C930D230DD30C8045B105B105E
:1000B000D204DD04E804F3045B10F7045B100505CB
:1000C0005B100F05190523055B105B105B103305F2
:1000D00040054D05F61AF81A311B311B311B311B37
:1000E000311B311B311B311B311B311BFE1A001B15
:1000F000021B041B061B081B0A1B0C1B311B101BBD
:10010000121B141B161B181B1A1B311B1C1B084A25
:10011000D73B3BCE016E84BCBFFDC12F3D6C74311B
:100120009ABD56833DDA3D00C77F11BED9E4BB4C72
:100130003E916BAAAABE000000803F05A84CCDB23C
:10014000D44EB93836A9020C50B9918688083CA61D
:10015000AAAA2ABE000000803F000D0A4772626C06
:1001600020312E3167205B27242720666F7220689C
:10017000656C705D0D0A00244E005B4F50543A00D0
:100180005B5645523A312E31672E3230313831319B
:1001900031323A005B544C4F3A005B4739323A00F7
:1001A0003330003238005B4700204700204D0020EC
:1001B000530020460020540033382E005B47433A5A
:1001C00047005B484C503A24242024232024472015
:1001D000244920244E2024783D76616C20244E78DA
:1001E0003D6C696E6520244A3D6C696E6520245320
:1001F0004C50202443202458202448207E202120B5
:100200003F206374726C2D785D0D0A00536C656538
:1002100070696E6700526573746F72696E672073E0
:1002200070696E646C6500526573746F72696E6795
:100230002064656661756C74730050676D20456E4F
:100240006400436865636B204C696D697473004397
:100250006865636B20446F6F720044697361626C00
:10026000656400456E61626C656400436175746924
:100270006F6E3A20556E6C6F636B6564002724487F
:10028000277C2724582720746F20756E6C6F636B52
:1002900000526573657420746F20636F6E74696EAD
:1002A0007565005B4D53473A00414C41524D3A0051
:1002B0007C413A007C4F763A007C57434F3A007CB1
:1002C000506E3A007C46533A007C42663A007C57B6
:1002D000506F733A007C4D506F733A00536C6565F4
:1002E0007000446F6F723A00436865636B00416C45
:1002F00061726D00486F6D65004A6F6700486F6CF2
:10030000643A0052756E0049646C65000D0A005B2A
:100310005052423A006572726F723A0000007A439E
:1003200000007A4300007A430000FA430000FA43D9
:100330000000FA4300A00C4700A00C4700A00C47A7
:10034000000048C3000048C3000048C30A00001969
:10035000010AD7233C6F12033B00007A44000000DF
:100360000000000000C8410000FA43FA00000080CD
:100370003F6F6B0D0A0011241FBECFEFD8E0DEBF28
:10038000CDBF27E0A0E0B1E001C01D92A136B207C9
:10039000E1F70E94D72B0C94703A0C940000EBE626
:1003A000F0E08081897E8083E8E6F0E080818E7FC6
:1003B0008083089584B1897E84B985B1866185B9C9
:1003C0008091700183FF0BC080916B0086618093E8
:1003D0006B008091680081608093680008950C94A0
:1003E000CF01F999FECF92BD81BD81E08FBB80B571
:1003F00008951F920F920FB60F9211242F933F93DF
:100400004F935F936F937F938F939F93AF93BF931C
:10041000EF93FF9380911A01813049F08091080792
:10042000811105C00E94042981E00E941D1DFF91D9
:10043000EF91BF91AF919F918F917F916F915F915C
:100440004F913F912F910F900FBE0F901F901895D5
:1004500093B196718091700186FD02C086E1982764
:10046000992349F091FB882780F992FD8260907171
:1004700019F08460089580E0089561E071E088E9F2
:1004800091E00C94361D9F92AF92BF92CF92DF9273
:10049000EF92FF920F931F93CF93DF935B018A013B
:1004A0007C01E40EF51EEC01912C6B01C81AD90AEF
:1004B000C6018C0F9D1FCE15DF0589F00E94F1014A
:1004C000911008C0292D990C330B232F221F2227AE
:1004D000221F01C021E0982E920E8993E9CFC50119
:1004E000800F911F0E94F10121E030E0981611F079
:1004F00020E030E0C901DF91CF911F910F91FF9073
:10050000EF90DF90CF90BF90AF909F900895F894B8
:10051000F999FECF92BD81BD81E08FBB80B5862762
:10052000482F082E000C550B262F30E024233523AE
:10053000232B39F06F3F19F060BD84E006C084E1E1
:1005400004C0882321F060BD84E28FBBF99A7894BF
:1005500008959F92AF92BF92CF92DF92EF92FF9257
:100560000F931F93CF93DF935C018A017B01E40E0D
:10057000F51EEB01912C6C01C61AD70ACE018C0D29
:100580009D1DCE15DF0589F0911008C0292D990C0D
:10059000330B232F221F2227221F01C021E0699144
:1005A000922E960E0E948702E9CF692DC501800F19
:1005B000911FDF91CF911F910F91FF90EF90DF90EE
:1005C000CF90BF90AF909F900C94870290911B01A9
:1005D000911107C086FF02C0439A01C04398109250
:1005E000250108952F923F924F925F926F927F92D2
:1005F0008F929F92AF92BF92CF92DF92EF92FF9233
:100600000F931F93CF93DF93CDB7DEB7CA54D109B1
:100610000FB6F894DEBF0FBECDBF8AE3E0ECF1E089
:10062000DF011D928A95E9F78BE0E0E8F1E0A1ECAB
:10063000B1E001900D928A95E1F780911107843223
:1006400011F00C947C1081E08093C1011092C201E2
:1006500083E08A8FB1E0BBA3212C312C1CA61BA602
:1006600010E01B8E1F8EEE24E394F12CEAE0AE2EF8
:10067000B12CF1E68F2EF3E09F2E8A8DE82FF0E06B
:10068000EF5EF84FD080DD2009F437C29FEB9D0D5F
:100690009A3110F00C944B108F5F8A8FBE016A5E06
:1006A0007F4FCE014A960E942829882311F40C948A
:1006B0004D104E885F88688C798CC301B2010E940E
:1006C000DB390E941937062F70E080E090E00E942D
:1006D0004A379B01AC01C301B2010E94A03520E062
:1006E00030E048EC52E40E94F8380E9465390E94DC
:1006F0001937CB01E7E4DE1629F0FDE4DF1609F433
:10070000EAC035C1083209F4C6C020F5043168F4E6
:10071000013108F08AC0043009F452C008F464C002
:100720000A3009F445C00C945B100C3109F440C048
:1007300050F4063110F00C945B1025E1201B20933F
:10074000C30126E0ADC00E3199F1063209F44CC068
:100750000C945B100D3309F498C0A8F4053381F1B3
:1007600040F40B3209F47AC0013309F477C00C94D9
:100770005B100C3310F00C945B106AEC600F60930C
:10078000C70129E08DC00C3538F40A3508F053C094
:10079000003581F10C945B100C3551F00F3510F0E1
:1007A0000C945B102EE5201B2093C20125E078C03D
:1007B000009731F42F8D21110C944F1031E03F8FB1
:1007C0000093C001202F2D7F2C3119F00C3509F03A
:1007D00064C0009721F00A9711F00C945B10600F31
:1007E0006093C00120E061C04F8D41110C944F1007
:1007F000A2E0AF8F0093C101063209F050C08431EE
:10080000910559F08E31910541F08832910529F01A
:100810008233910511F00C945B10B5010E940D3AE2
:1008200066576093C10121E040C06FEE600F609396
:10083000C50122E035C0892B31F466EA600F609370
:10084000C40123E032C06A30710511F00C945B10D2
:100850000A3511F40C945B1024E027C0BF8DB11150
:100860000C944F10013331F41092C60128E0E3E0FC
:10087000EF8F1BC00A9711F00C945B10F1E0F0931E
:10088000C60128E033E03F8F10C0892B11F00C9493
:100890005B102AE00AC027E003C020E001C021E08D
:1008A000892B19F087E10C948310C70102C0880FCF
:1008B000991F2A95E2F72BA53CA528233923232B42
:1008C00019F085E10C948310ABA5BCA5A82BB92B1E
:1008D000BCA7ABA7D2CE892B29F7063018F403307A
:1008E00058F016C0083010F40C945B100A30F0F089
:1008F0000E3159F00C945B10002319F0013011F106
:1009000004C0B3E0B093C8011DC00093C8011AC071
:10091000043021F0053031F080E101C080E28093A5
:10092000CA0102C01092CA018CE00DC0093031F03A
:100930008091C90180648093C90102C01092C901ED
:100940008DE001C08BE0F70102C0EE0FFF1F8A951A
:10095000E2F72BA53CA52E233F23232B09F0B1CF93
:100960002BA53CA52E2B3F2B3CA72BA786CE8D2D50
:10097000DD0C990BAA0BBB0BFC01E654F109E53128
:10098000F10510F00C945B10EB5AFF4F0C94433AB6
:100990004092CC015092CD016092CE017092CF0175
:1009A00080E087C04092D0015092D1016092D20184
:1009B0007092D301116081E07CC04092D4015092CA
:1009C000D5016092D6017092D701126082E071C0A9
:1009D0004092D8015092D9016092DA017092DB0105
:1009E000146083E066C00093DC0184E062C0C30150
:1009F000B2010E9412376093DD017093DE01809393
:100A0000DF019093E00185E054C04092E1015092F3
:100A1000E2016092E3017092E40186E04AC04092F4
:100A2000E5015092E6016092E7017092E80187E0EB
:100A300040C04092E9015092EA016092EB0170924D
:100A4000EC0188E036C020E030E04FE753E4C3011A
:100A5000B2010E94B838181614F40C945110009387
:100A6000ED0189E026C04092EE015092EF016092C4
:100A7000F0017092F1013B8D31603B8F8AE019C02B
:100A80004092F2015092F3016092F4017092F501EC
:100A90004B8D42604B8F8BE00CC04092F601509220
:100AA000F7016092F8017092F9018B8D84608B8F51
:100AB0008CE06701082E02C0CC0CDD1C0A94E2F722
:100AC000960122213321232B11F00C945310D401D1
:100AD00002C0B595A7958A95E2F7A0FF0BC020E06C
:100AE00030E0A901C301B2010E94963687FF02C01F
:100AF0000C9455102C283D28C0CDBB8DBB2329F06C
:100B0000EF8DE11102C0F2E0FF8F25FE0FC0809152
:100B1000DD019091DE01A091DF01B091E00181380B
:100B20009649A849B10514F00C9457103BA1332302
:100B300029F020FC02C00C94611018C08091C20101
:100B4000813071F44F8D4230E1F58091C1018035E3
:100B5000C1F18823B1F120FC02C00C94611031C0B6
:100B60008091810181112DC020FE1BC08091C301A5
:100B7000813039F523E333E34BEC51E46091CC0150
:100B80007091CD018091CE019091CF010E94F838F3
:100B90006093CC017093CD018093CE019093CF01EF
:100BA00010C080918F0190919001A0919101B0911E
:100BB00092018093CC019093CD01A093CE01B0938C
:100BC000CF0130FC10C080918B0190918C01A091DD
:100BD0008D01B0918E018093E9019093EA01A09379
:100BE000EB01B093EC018091C001843039F426FC14
:100BF00003C08CE10C948310E89426F88091C50121
:100C0000882369F0813029F48FAF1DAE92E09BAF4D
:100C10000BC01FAEA2E0ADAFB1E0BBAF05C0E2E0DC
:100C2000EFAFF1E0FDAF1BAE8091C301813021F049
:100C30002F8D2330C9F52FC060ECC62E61E0D62E73
:100C4000E12CF12C3B8DA32EB12CC5010E2C02C042
:100C5000959587950A94E2F780FF12C023E333E36A
:100C60004BEC51E4D6019E966D917D918D919C91B6
:100C7000D1970E94F838F60166A777A780AB91ABB1
:100C8000FFEFEF1AFF0A24E0C20ED11C33E0E31697
:100C9000F104D9F6CDCF8091C601813029F44B8D76
:100CA000443011F00C9459108CE0E4EAF1E0DE01DC
:100CB000119601900D928A95E1F78BA59CA591FD67
:100CC00008C00091C0010A30C9F00C3509F4B3C066
:100CD0001EC18091C701873018F08DE10C948310FC
:100CE00090918601891769F3BE016F5F7F4F0E9463
:100CF000421A882311F40C946F10E3CF9B8D91114D
:100D000003C08AE10C948310C10180759927892B57
:100D100009F46FCF6091E1017091E2018091E301EC
:100D20009091E4010E94DB390E9419376730A8F6E0
:100D30008091DC01843141F0823011F00C945B1021
:100D400027FE02C00C945B10AFEA2A22662319F03A
:100D5000615069A703C0B091C701B9A760ED71E008
:100D600089A50E94421A882311F40C946F100091F7
:100D7000DC014090BC015090BD016090BE017090BC
:100D8000BF0140ECE42E41E0F42E50E8A52E51E0E6
:100D9000B52EC12CD12CEB8D8E2E912CC4010C2C98
:100DA00002C0959587950A94E2F780FF35C004311B
:100DB00051F5D501D0962D913D914D915C91D397F0
:100DC00058966D917D918D919C915B970E94A03575
:100DD000F70126A537A540A951A90E94A035D70142
:100DE00050966D937D938D939C935397B2E0CB1265
:100DF00013C0A30192010E94A035F701608B718B93
:100E0000828B938B09C0F70186A597A5A0A9B1A9EC
:100E1000808B918BA28BB38BFFEFCF1ADF0A24E07C
:100E2000E20EF11C34E0A30EB11C43E0C416D10461
:100E300009F0B4CF3FC18B8D882309F462CF409075
:100E4000BC015090BD016090BE017090BF0120E8D0
:100E5000822E21E0922EDE0111967D0130ECC32E10
:100E600031E0D32EA12CB12CE82FF0E0F8A7EFA3AE
:100E70008FA198A50A2C02C0959587950A94E2F750
:100E800080FF29C0D7012D913D914D915C91F401D6
:100E9000608D718D828D938D0E94A035D6019E96B6
:100EA0002D913D914D915C91D1970E94A035F60115
:100EB00066A777A780AB91ABF2E0AF1216C0A30193
:100EC00092010E94A035D6019E966D937D938D93DD
:100ED0009C93D1970AC0F40180A991A9A2A9B3A9B2
:100EE000F60186A797A7A0ABB1ABFFEFAF1ABF0A79
:100EF00024E0820E911C34E0E30EF11C44E0C40EA9
:100F0000D11C83E0A816B10409F0B2CFD2C09F8DE6
:100F1000933069F40E3109F494C0053309F4C3C069
:100F20000C3109F0C6C060ED71E086E08DC0AB8D7C
:100F3000AA2381F3B091C401BFA34090BC0150909B
:100F4000BD016090BE017090BF0180E8A82E81E0D5
:100F5000B82E90ECE92E91E0F92EFE0131964F016A
:100F6000C12CD12C2A2F30E03AA729A789A59AA510
:100F70000C2C02C0959587950A94E2F780FD0BC072
:100F8000F501808D918DA28DB38DF70186A797A76E
:100F9000A0ABB1AB44C0053309F441C0FFA1F111CE
:100FA0002BC0D501D0962D913D914D915C91D39759
:100FB000F40160817181828193810E94A135D70102
:100FC0009E962D913D914D915C91D1970E94A135B6
:100FD000F70166A777A780AB91ABF2E0CF121FC0F5
:100FE000A30192010E94A135D7019E966D937D9336
:100FF0008D939C93D19713C0F501208D318D428D37
:10100000538DD7019E966D917D918D919C91D19735
:101010000E94A135F70166A777A780AB91ABFFEFE0
:10102000CF1ADF0A24E0A20EB11C34E0E30EF11C5B
:1010300044E0840E911C83E0C816D10409F096CFD9
:1010400069CF60ED71E087E00E94421A882311F4B5
:101050000C946F109B8D911103C019A61F8E2AC08E
:10106000A0E8B1E0E0ECF1E080E090E04B8D242FCF
:1010700030E0A901082E02C0559547950A94E2F781
:1010800040FD0AC058964D915D916D917C915B97A2
:10109000408B518B628B738B019614963496833000
:1010A000910539F706C08091C101823010F00C948F
:1010B0005D1019A68091C1018FA3803529F49B8D05
:1010C00091110C945F107AC2AF8DA23009F076C2F4
:1010D000BFA1B11104C0EB8DE11170C22AC020E0A4
:1010E00030E0A9016091CC017091CD018091CE01D9
:1010F0009091CF010E949636882309F4E2C7FFA1A0
:10110000FC3809F445C240F4F230A9F0F330B1F0F4
:10111000F13009F053C20AC02FA12E3809F438C2A9
:1011200008F433C22F3809F430C248C23B8D311164
:1011300045C21F8E43C24BA144604BA38B8D8823B5
:1011400009F4DFCDBBADAB2FB0E0B8ABAFA7FDADC1
:10115000EF2FF0E0FCABEBAB81E090E07C010BAC5F
:1011600002C0EE0CFF1C0A94E2F70DAC02C0880F1F
:10117000991F0A94E2F7E82AF92A2B8D822F90E032
:101180008E219F21892B09F49EC7FD01EE0FFF1FC1
:10119000EE0FFF1FE054FE4FAA0FBB1FAA0FBB1F8D
:1011A000A856BE4F2D913D914D915C9166A577A5B6
:1011B00080A991A90E94A0352B013C01EBA9FCA9B3
:1011C000EE0FFF1FEE0FFF1FE054FE4FABA9BCA9AF
:1011D000AA0FBB1FAA0FBB1FA856BE4F2D913D9152
:1011E0004D915C9166A577A580A991A90E94A03533
:1011F0004B015C01610130E8C322DD2427FEF5C00C
:10120000E89427F84CE050E06EEE71E088E991E058
:101210000E94633A892B11F481E275C78091C30162
:101220008130B1F423E333E34BEC51E46091E50109
:101230007091E6018091E7019091E8010E94F838F1
:101240006093E5017093E6018093E7019093E801D4
:101250008091E5019091E601A091E701B091E8014C
:101260008FAB98AFA9AFBAAFA3019201C301B2018E
:101270000E94F83827966CAF7DAF8EAF9FAF27974F
:10128000A5019401C501B4010E94F8382B966CAFFA
:101290007DAF8EAF9FAF2B9720E030E040E850E469
:1012A0006FA978AD89AD9AAD0E94F8382FA938ADF5
:1012B00049AD5AAD0E94F83827962CAD3DAD4EADE4
:1012C0005FAD27970E94A0352B962CAD3DAD4EAD5E
:1012D0005FAD2B970E94A0356B017C0120E030E0D0
:1012E000A9010E94963687FDF0C6C701B6010E948B
:1012F00097396B017C012B962CAD3DAD4EAD5FADAA
:101300002B9727966CAD7DAD8EAD9FAD27970E9434
:10131000A1350E9497399B01AC01C701B6019058D5
:101320000E94A0366B017C019FA1933021F4F7FA53
:10133000F094F7F8F09420E030E0A9016FA978ADBF
:1013400089AD9AAD0E94963687FF11C0F7FAF094E6
:10135000F7F8F0948FA998ADA9ADBAADB0588093C5
:10136000E5019093E601A093E701B093E8010FA592
:1013700018A9000F111F000F111F00531E4FA701C6
:101380009601C501B4010E94F8389B01AC01C3016C
:10139000B2010E94A03520E030E040E05FE30E940F
:1013A000F838D8016D937D938D939C9313970BA977
:1013B0001CA9000F111F000F111F00531E4FA70182
:1013C0009601C301B2010E94F838A50194010E9460
:1013D000A13520E030E040E05FE30E94F838F801FA
:1013E0006083718382839383E9C0212F30E038AF1B
:1013F0002FABE222F322EF2809F469C631EF232252
:101400008091C301813009F47BC0EFA5F8A9EE0FEC
:10141000FF1FEE0FFF1FE053FE4FC080D180E28020
:10142000F380A7019601C301B2010E94A0352B01F0
:101430003C01EBA9FCA9EE0FFF1FEE0FFF1FE053CD
:10144000FE4F80819181A281B3818FA798ABA9AB18
:10145000BAAB9C01AD01C501B4010E94A0354B019E
:101460005C01A3019201C301B2010E94F8382B0173
:101470003C01A5019401C501B4010E94F8389B010B
:10148000AC01C301B2010E94A1350E9497394B0102
:101490005C01A7019601C701B6010E94F8386B01F3
:1014A0007C012FA538A949A95AA9CA01B9010E94EE
:1014B000F8389B01AC01C701B6010E94A1350E941A
:1014C00097396B017C016093E5017093E60180938D
:1014D000E7019093E8019B01AC01C501B4010E94B2
:1014E000A0354B015C01E894B7F82AE037ED43EAF8
:1014F0005BE3C501B4010E94B83818164CF15EC018
:1015000000EC11E08FA998AD0C2C02C09595879541
:101510000A94E2F780FF12C023E333E34BEC51E47B
:10152000D80150966D917D918D919C9153970E9419
:10153000F838F801608B718B828B938BFFEFCF1A99
:10154000DF0A0C5F1F4F23E0C216D104D9F65DCF2E
:1015500020E030E040E05FE3C501B4010E94B8380C
:1015600018160CF459CE2FE632E143E85AE3C701CE
:10157000B6010E94F8389B01AC01C501B4010E947C
:10158000B83818160CF448CE19C03BA130613BA303
:101590008FA18E58823018F44BA148604BA38B8DDD
:1015A000882309F4AECB4CE050E06EEE71E088E9A0
:1015B00091E00E94633A892B09F42ECE2BA1217071
:1015C0009BA190FF03C0C1018E7D03C0C1018E7D30
:1015D0009C7FAF8DA111937E892B09F07AC58E0176
:1015E000035F1F4F89E0F80111928A95E9F72223E2
:1015F00009F44BC08BA59CA5867B892B09F06BC594
:101600008091C001853311F0811165C580918B01F6
:1016100090918C01A0918D01B0918E01898B9A8B54
:10162000AB8BBC8B9091890180918801892B409173
:10163000CC015091CD016091CE017091CF014D87C9
:101640005E876F87788B84608D8B8091700185FFBA
:1016500006C08EEE91E00E94803181113EC5B80136
:101660008EEE91E00E943D3580911A01811139C5BD
:101670000E945627892B09F434C580E280931A0111
:101680000E94BB1D0E940E192CC580917001F09024
:10169000890181FF26C08FA18150833018F0FBA102
:1016A000F064FBA32B8D222339F03F8D323021F4DF
:1016B0004BA140684BA315C080E1F81212C0809185
:1016C000800181509BA19074833030F4992349F0BC
:1016D0009BA190629BA305C0911103C0ABA1A06226
:1016E000ABA38091DD019091DE01A091DF01B0916B
:1016F000E0018093940190939501A0939601B0939B
:1017000097018091C20180938101882311F088E0C4
:101710008D8B8091CC019091CD01A091CE01B091A3
:10172000CF0180938F0190939001A0939101B0938A
:1017300092018D879E87AF87B88B8090E90190904A
:10174000EA01A090EB01B090EC01A5019401609139
:101750008B0170918C0180918D0190918E010E947E
:101760009636BBA1B074EB2E811103C0EBA1E5FF4F
:1017700020C0FF2071F0FBA1F7FD0BC0EE2021F08F
:1017800040E050E0BA0102C0B501A4018F2D0E94D3
:1017900038318091E9019091EA01A091EB01B0917B
:1017A000EC0180938B0190938C01A0938D01B093F9
:1017B0008E01E1100CC080918B0190918C01A09161
:1017C0008D01B0918E01898B9A8BAB8BBC8B8091F4
:1017D000ED01809393018091CA019091890198173E
:1017E00051F049895A896B897C890E9438318091EE
:1017F000CA01809389019D8980918901892B8D8BF4
:10180000F090C901809188018F1569F080911A01CB
:10181000823029F00E9466278F2D0E94E602809177
:10182000C901809388019D8980918801892B8D8BC6
:101830008091C001843099F4C090E101D090E20120
:10184000E090E301F090E40180911A01823039F0D8
:101850000E94662740E0C701B6010E94D52880910A
:10186000C501809384018091C301809382012F8DF3
:10187000233071F58091C60180938501811108C0E4
:101880001092F6011092F7011092F8011092F901EE
:10189000C090F601D090F701E090F801F090F901C6
:1018A000A70196016091BC017091BD018091BE01BC
:1018B0009091BF010E949636882351F0C092BC01DE
:1018C000D092BD01E092BE01F092BF010E94BB31F7
:1018D0008091C70190918601981769F080938601E5
:1018E0008CE0FE013196A4EAB1E001900D928A9558
:1018F000E1F70E94BB318091C40180938301809104
:10190000C0018632F1F138F48C3109F18E31F9F0F1
:101910008A3069F04FC08C35D1F1863609F441C068
:10192000883209F047C068E971E087E02DC060EDBA
:1019300071E089A50E942E1A8091860139A538137D
:1019400039C08CE0E0EDF1E0A4EAB1E025C08D897A
:1019500081608D8B4F8D442329F0B8018EEE91E08C
:101960000E943D35B80180ED91E00E943D358CE04C
:10197000E0EDF1E0A8E9B1E001900D928A95E1F780
:1019800019C068E971E086E00E942E1A13C08CE04D
:10199000EEEEF1E0A0EBB1E001900D928A95E1F757
:1019A00007C08CE0E0EBF1E0DF011D928A95E9F7DA
:1019B0000E94BB318091C10180938001803509F480
:1019C0001CC3BF8DB23009F018C3813021F4BE01B1
:1019D000635F7F4F06C0811109C08D8981608D8B47
:1019E000B8018EEE91E00E943D35FEC282508230F9
:1019F00008F093C28091E5019091E601A091E70182
:101A0000B091E8018F8F98A3A9A3BAA3ABAD94E0DE
:101A1000A99F70011124F701E856FE4FF8A7EFA324
:101A2000970120533E4F3AA729A7D9014D905D90C9
:101A30006D907C902081318142815381C301B2013C
:101A40000E94A1356BA77CA78DA79EA7EDADB4E042
:101A5000EB9F80011124980128563E4F3CAF2BAFDD
:101A6000C80180539E4F9EAF8DAFDC018D909D903D
:101A7000AD90BC90F9012081318142815381C50133
:101A8000B4010E94A1356FA778AB89AB9AAB77FA06
:101A9000709477F87094D501C401B0588B8F9C8FE7
:101AA000AD8FBE8FF701E251FE4F2BA53CA54DA592
:101AB0005EA560817181828193810E94A0356B0156
:101AC0007C01F801E251FE4F2FA538A949A95AA976
:101AD00060817181828193810E94A0354B015C01FC
:101AE000A7019601C301B2010E94F8386BAB7CAB31
:101AF0008DAB9EABA50194016B8D7C8D8D8D9E8DE4
:101B00000E94F8389B01AC016BA97CA98DA99EA904
:101B10000E94A1356BAB7CAB8DAB9EABA501940154
:101B2000C301B2010E94F8384B015C01A701960184
:101B30006B8D7C8D8D8D9E8D0E94F8389B01AC0144
:101B4000C501B4010E94A0352BA93CA94DA95EA9ED
:101B50000E9420366B017C019BA192FF13C02DEBEC
:101B600037E346E055EBC701B6010E94B83887FD60
:101B70001DC02BED3FE049EC50E4C701B6010E94C7
:101B8000A03512C02DEB37E346E055E3C701B6019F
:101B90000E949636181654F02BED3FE049EC50E4C5
:101BA000C701B6010E94A1356B017C0180906401E0
:101BB00090906501A0906601B09067012F8D38A1CB
:101BC00049A15AA1CA01B9010E94A135A5019401F8
:101BD0000E94A035A50194010E94F8380E9497390F
:101BE0004B015C0120E030E040E05FE3C701B6015B
:101BF0000E94F8382F8D38A149A15AA10E94F838C7
:101C00009F77A50194010E94A0360E9485370E940B
:101C100019377CAB6BABDB01AB2B09F4D8CE1D893C
:101C20004B01A12CB12C13FF12C0C501B4010E94BD
:101C300048379B01AC016D857E858F8598890E9410
:101C4000F8386D877E878F87988B177F1D8BC5012E
:101C5000B4010E9448374B015C019B01AC01C701F4
:101C6000B6010E94A0366BA37CA38DA39EA3EFAD0B
:101C7000B4E0EB9FC00111248C0108561E4FFC01FB
:101C8000E251FE4FD8012D913D914D915C916081C3
:101C90007181828193810E94A035A50194010E94E7
:101CA000A03627966CAF7DAF8EAF9FAF27972BA145
:101CB0003CA14DA15EA1CA01B9010E94F8389B0167
:101CC000AC0160E070E080E090E40E94A0356B0120
:101CD0007C012BEA3AEA4AE25EE36BA17CA18DA18A
:101CE0009EA10E94F8384B015C0120E030E040E802
:101CF00050E4C701B6010E94A1359B01AC01C501AA
:101D0000B4010E94F8386FAB78AF89AF9AAF20E08A
:101D100030E040E05FE3C701B6010E94F838239647
:101D20006CAF7DAF8EAF9FAF23971F8E222423947D
:101D3000312CEBA9FCA9E215F30509F448CEBF8DBF
:101D4000BC3008F044C02B8D3C8D4D8D5E8D2396AC
:101D50006CAD7DAD8EAD9FAD23970E94F8386B01C1
:101D60007C01A30192016FA978AD89AD9AAD0E9463
:101D7000F838A70196010E94A1357B016C01A301EF
:101D8000920123966CAD7DAD8EAD9FAD23970E94E1
:101D9000F8384B015C012B8D3C8D4D8D5E8D6FA90C
:101DA00078AD89AD9AAD0E94F8389B01AC01C501B0
:101DB000B4010E94A0352B013C01EF8DEF5FEF8F46
:101DC000470156018B8E9C8EAD8EBE8E65C0B101D3
:101DD00080E090E00E9448372BA13CA14DA15EA17C
:101DE0000E94F8386B017C010E949B366B8F7C8FC0
:101DF0008D8F9E8FC701B6010E9489394B015C010E
:101E0000A9A5BAA5CD90DD90ED90FC90F7FAF094DD
:101E1000F7F8F094ADADBEAD8D919D910D90BC9154
:101E2000A02D8F8F98A3A9A3BAA3A70196016B8DAC
:101E30007C8D8D8D9E8D0E94F8382B013C012F8D5D
:101E400038A149A15AA1C501B4010E94F8389B01EB
:101E5000AC01C301B2010E94A1352B013C01A701D5
:101E60009601C501B4010E94F8386B017C012F8DE9
:101E700038A149A15AA16B8D7C8D8D8D9E8D0E94BC
:101E8000F8389B01AC01C701B6010E94A0356B8FE9
:101E90007C8F8D8F9E8F1F8EA30192016BA57CA5D9
:101EA0008DA59EA50E94A135EFA1F8A56083718341
:101EB000828393832B8D3C8D4D8D5E8D6FA578A98C
:101EC00089A99AA90E94A135ABADBCAD6D937D9354
:101ED0008D939C93139727962CAD3DAD4EAD5FAD82
:101EE0002797F80160817181828193810E94A135D9
:101EF000D8016D937D938D939C931397BE01635F7F
:101F00007F4F88E991E00E943D3580911B0181114E
:101F10006BC0BFEF2B1A3B0A0CCF8D8984608D8B71
:101F200080911A01823009F45FC00E946627809177
:101F30001B01811162C0FBA1F071FF2E10921F01E5
:101F40002BA123FB882780F90E94D02586B18072BF
:101F500090910001891749F084E00E941D1D0E94A4
:101F6000351580E00E94D02548C0B8018EEE91E082
:101F70000E943D3581E08093190182E00E942D1D71
:101F80000E94351580911B01811137C080911A0183
:101F90008111F6CF80911901813081F4FF2051F039
:101FA0008CE0E1E0F1E0ADE0B1E001900D928A95C6
:101FB000E1F707C085E00E941D1D03C081E080930A
:101FC0001F011092190180E00E94D0250E94351552
:101FD0000E949D250E9477270E94D2260E9456319A
:101FE00080911F0181118CC08CE0EEEEF1E0A8E938
:101FF000B1E001900D928A95E1F78091C80180933C
:102000008701882309F47FC00E9466278091870199
:1020100090911A01833041F49230D1F188E00E940E
:102020002D1D0E94351534C081E0809380011092EF
:102030008401109283011092810110928601109206
:1020400089011092880184E6809321018093220106
:1020500080932301923091F064EA71E080E00E9465
:10206000421A8823E1F10E94BB3140E050E0BA01FE
:1020700080E00E94C31980E00E94E60283EA92E0B9
:102080000E94C3268AE392E00E94C3260E94EE10BB
:10209000109287012FC081E036C082E034C088E111
:1020A00032C086E230C089E12EC084E02CC08BE1D2
:1020B0002AC085E228C084E126C08EE124C08FE1D9
:1020C00022C086E120C080E21EC082E21CC083E202
:1020D0001AC084E218C080E116C08FE014C087E007
:1020E00012C08CE0EEEEF1E0A8E9B1E001900D92B3
:1020F0008A95E1F780E007C01A8E1BA20C942C038E
:102100000E943D027ACFC65BDF4F0FB6F894DEBF68
:102110000FBECDBFDF91CF911F910F91FF90EF9038
:10212000DF90CF90BF90AF909F908F907F906F90F7
:102130005F904F903F902F9008950F931F93CF93F0
:102140008C01C0E0F80161917191819191918F01B1
:102150000E948E26C23019F08CE20E946C1BCF5F69
:10216000C33081F7CF911F910F9108958CE093E0D8
:102170000C94C326CF92DF92EF92FF92CF93DF931E
:10218000D82F6A017B01C22F84E20E946C1B8D2F25
:102190000E949D268DE30E946C1B4C2FC701B60147
:1021A0000E94E225DF91CF91FF90EF90DF90CF90DA
:1021B0000C94B610CF93DF93D82FC62F84E20E94E1
:1021C0006C1B8D2F0E949D268DE30E946C1B8C2F13
:1021D0000E949D26DF91CF910C94B6108DE50E9450
:1021E0006C1B0C94B6103F924F925F926F927F924D
:1021F0008F929F92AF92BF92CF92DF92EF92FF9217
:102200000F931F93CF93DF93CDB7DEB7A4970FB68D
:10221000F894DEBF0FBECDBF10910807112391F1D6
:1022200081E080931A0189EA92E00E94C326812FFF
:102230000E949D260E94B61085EF91E0019739F02B
:10224000EFE9FFE03197F1F700C00000F7CF115040
:10225000123030F08FB7F894109208078FBF12C079
:1022600083EA92E00E94C32681E992E00E94C3269D
:102270000E94EE1080E10E94231D8091070784FFD9
:10228000FCCFE8CF10910707112309F4BBC214FF5C
:1022900004C081E080931B01D0C310FFBFC18CE05C
:1022A000E1E0F1E0DE01599601900D928A95E1F7A7
:1022B000BE01675E7F4FCE010D960E94361D8CE3F6
:1022C0000E946C1B80911A018830E1F058F4813033
:1022D00099F1A8F0823099F1843009F043C084EF7D
:1022E00092E03EC0803229F118F4803171F03AC09A
:1022F000803441F18038B1F58CED92E031C087E057
:1023000093E02EC083E093E02BC080911C0187FDF9
:1023100010C08DEF92E00E94C32680911C0180FFC7
:1023200006C080E31AC082FF17C085FFFACF81E3A1
:1023300014C089EF92E014C08EEE92E011C088EED6
:1023400092E00EC082EE92E00E94C32680911C01B2
:1023500083FFE9CF83E301C082E30E946C1B02C0CC
:102360000E94C32680915F01F82FF170BF2E80FF7D
:1023700007C080912601882319F085ED92E053C0B3
:102380004090BC015090BD016090BE017090BF01B3
:1023900054EA852E51E0952E9E012F5F3F4F790123
:1023A000CE010D966C0100E0F40161917191819173
:1023B00091914F0120853185428553850E94A13539
:1023C000F7016083718382839383023061F4A301F8
:1023D00092010E94A135F701608371838283938308
:1023E000BB2019F0CACFB11011C0F7012081318193
:1023F00042815381F60160817181828193810E94C3
:10240000A035F60160837183828393830F5FF4E0CC
:10241000EF0EF11C24E0C20ED11C033029F6B110DE
:10242000ACCF8EEC92E00E94C326CE010D960E94A6
:102430009D1080915F0181FF1FC089EC92E00E9496
:10244000C3269091500680912F03981710F0815F5A
:1024500001C08150891B0E949D268CE20E946C1B4A
:102460008091970290919802981710F0805801C0BF
:102470008150891B0E949D2684EC92E00E94C32615
:1024800080911A018C7749F06091EE067091EF0609
:102490008091F0069091F10603C060E070E0CB01FE
:1024A0000E947F268CE20E946C1B60912701709134
:1024B00028018091290190912A0140E00E94E225A3
:1024C0000E942802F82E0E94721D082F86B1982FB4
:1024D000907280910001E92EE8268F2D802B8E29A5
:1024E00059F18FEB92E00E94C326EE2019F080E5AF
:1024F0000E946C1BFF2079F0F0FE03C088E50E946B
:102500006C1BF1FE03C089E50E946C1BF2FE03C048
:102510008AE50E946C1B002379F000FF03C082E56E
:102520000E946C1B01FF03C088E40E946C1B02FF29
:1025300003C083E50E946C1B80912601882321F053
:1025400081508093260118C080911A018C7711F078
:102550008DE101C089E080932601809125018111E0
:1025600003C081E08093250189EB92E00E94C3269D
:10257000CE0101960E949D1000912501002321F0BB
:1025800001500093250142C080911A018C7711F00F
:1025900083E101C089E08093250184EB92E00E94F1
:1025A000C326809121010E949D268CE20E946C1B13
:1025B000809122010E949D268CE20E946C1B8091DA
:1025C00023010E949D268091B00087FF05C02D9BAE
:1025D00002C002E001C001E0439B03C040E4F42ECE
:1025E00003C0002399F0F12C80EB92E00E94C326F7
:1025F000002339F0013011F483E501C083E40E9427
:102600006C1BFF2019F086E40E946C1B8EE30E9475
:102610006C1B0E94B61081E00E94231D812F887ED2
:1026200009F467C080911A01982F937009F050C087
:102630008872A1F080911C01807C81F40E94792530
:1026400082E080931E0180911A01803239F417FDD7
:10265000F2C180911C01806880931C0180911A0155
:10266000811103C091E090931C0116FF07C085FD06
:1026700005C090911C01906490931C0113FF05C04C
:10268000807E19F480E180931A0115FF21C083EA4E
:1026900092E00E94C3268FE492E00E94C3260E942B
:1026A000EE1080911C0187FD0EC090911A019034AC
:1026B00039F483FFBCC1837E826080931C01B7C163
:1026C000903809F0B4C180911C01806280931C0194
:1026D00017FF0CC080911A01813029F480911C01F0
:1026E000856080931C0180E880931A0188EE0E9427
:1026F000231D11FF44C0812F8876F1F580911A01C6
:10270000803471F480911C0185FD0AC084FF03C0F0
:1027100010921A0105C082FF03C0886080931C01DB
:1027200080911A01882381F084FF26C090911C01BA
:1027300090FF22C0803141F480912401882321F050
:1027400088608093240118C010921E010E945627B1
:10275000892B71F080911C0186FD0AC010921C012A
:1027600088E080931A010E94BB1D0E940E1904C0CC
:1027700010921C0110921A0182E00E94231D12FF88
:1027800041C080911A01807D90911C018823D9F06D
:1027900080911D01811117C097FD15C00E947925F8
:1027A00080912F0380932E030E94882780911E0121
:1027B00081FF05C090911C01916090931C01897F5D
:1027C00080931E011CC097FF0AC010921E010E9438
:1027D00077270E949D250E943D020E94D22680916B
:1027E0001C0185FF08C08F77816080931C0180E405
:1027F00080931A0104C010921C0110921A0184E007
:102800000E94231D90910907992309F4ABC08FB74B
:10281000F894109209078FBF4091210190FD02C0EA
:10282000842F01C084E691FD865F92FD8A5093FD5E
:102830008F5F94FD8150893C08F088EC8A3008F461
:102840008AE03091220195FD02C0232F01C024E6C9
:1028500096FD22E397FD29E1481303C0231709F4ED
:1028600081C08093210120932201109225011091B3
:102870002F033090500689E9D82E96E7E92E26E9F5
:10288000F22E0EE732E3432E131509F457C0812EC2
:10289000912C489CC001499C900D1124FC01E05DE5
:1028A000FC4F5F01CF010E94E326562E672E782E43
:1028B000C92E2D2D3E2D4F2D502F0E94B8381816A1
:1028C0004CF42D2D3E2D4F2D502F6D2D7E2D8F2D07
:1028D000902F08C0252D362D472D5C2D652D762D8A
:1028E000872D9C2D0E94F838F501668B778B808FA1
:1028F000918F489CC001499C900D11249C01205D42
:102900003C4F7901F90182A093A0A4A0B5A0A50134
:10291000940166897789808D918D0E94B838181648
:102920002CF4F701868A978AA08EB18E1F5F103132
:1029300009F410E0D52C73010C2DA6CF8D2D9E2D02
:10294000AF2DB02F8093120290931302A093140224
:10295000B09315020E94792580912F0380932E0356
:102960000E94882710910A07112309F459C08FB7D4
:10297000F89410920A078FBF9091230110FD02C0B6
:10298000892F01C084E611FD865F12FD8A5013FD78
:102990008F5F14FD8150893C08F088EC8A3008F480
:1029A0008AE09817D1F08093230180911A01811158
:1029B0000DC040918B0150918C0160918D017091FF
:1029C0008E01809189010E94C31905C080911E016A
:1029D000886080931E011092250180911A0115FFD5
:1029E0000DC0803159F490912401911102C092E000
:1029F00003C090FF03C0946090932401107C81F089
:102A0000882311F0887361F01091880116FF02C0CD
:102A10001F7B01C01064812F0E94E6021093880181
:102A200080911A018C7F49F00E94BB1D06C080E492
:102A300080931A0148CE80E218CEA4960FB6F8947F
:102A4000DEBF0FBECDBFDF91CF911F910F91FF90E1
:102A5000EF90DF90CF90BF90AF909F908F907F903E
:102A60006F905F904F903F900895CF92DF92EF92DA
:102A7000FF921F93CF93DF930E94F31080911C016C
:102A8000882309F4FEC00E945627009771F4C09174
:102A9000890180918801C82BC0908B01D0908C0156
:102AA000E0908D01F0908E010EC0FC01C189C073D1
:102AB000439B02C020E401C020E0C22BFC01C6A45D
:102AC000D7A4E0A8F1A88091700181FF03C080E243
:102AD0000E940B1DDC2FD07311E0C07C80911C0183
:102AE000882309F4CEC090911B019111CAC080FFC8
:102AF000C5C090911A01292F207C09F474C082FD71
:102B000012C01092240140E050E0BA0180E00E941F
:102B1000C31980E00E94E60280911C018D7F8460D1
:102B200080931C01ABC09038E1F483EA92E00E94EC
:102B3000C3268CE092E00E94C3260E94EE1040E083
:102B400050E0BA0180E00E94C31980E00E94E602D2
:102B50000E94901680911B01811193C00E94F31076
:102B6000F9CF903419F48F7D80931C0180911C0162
:102B700083FF84C0909189019923C1F081FD16C023
:102B80008091700181FF06C080911E018860809352
:102B90001E010CC0B701A6018D2F0E94C31941E090
:102BA00060E070E080E890E40E94D5288091880180
:102BB000882371F080911C0181FD0AC08C2F0E9436
:102BC000E60241E060E070E080E89FE30E94D528E3
:102BD00080911C0181FD52C0806180931C0182E0C4
:102BE0000E942D1D4BC0809124018823C9F181FFD3
:102BF0000DC0809189018823B1F040E050E0BA0116
:102C000080E00E94C3191093240138C08C70B1F188
:102C10008091890181110AC08091240183FF03C042
:102C200082E00E942D1D1092240128C083EA92E0C8
:102C30000E94C32685E192E00E94C3260E94EE1006
:102C40008091700181FF06C080911E018860809391
:102C50001E01E2CFB701A6018D2F0E94C319DCCF60
:102C600080911E0183FF0AC0B701A6018D2F0E942B
:102C7000C31980911E01877F80931E010E94F3106B
:102C80002DCFDF91CF911F91FF90EF90DF90CF90EC
:102C900008950E945627892B19F082E00C942D1D6F
:102CA00008958093B300811104C08091B0008F77A4
:102CB00003C08091B00080688093B0000895809137
:102CC0005C01682F20915D01422F982F917080FD4B
:102CD00094E0822F817020FD80E261FD986041FDCB
:102CE000806462FD906142FD806890930803809348
:102CF000090308951F920F920FB60F9211248F931C
:102D00009F938BB1909108039C71837E892B8BB923
:102D100015BC9F918F910F900FBE0F901F9018952B
:102D200080916F008D7F80936F0080918100887FFC
:102D300081608093810010920A0380915E019091DE
:102D40001A018F3F39F420910807211103C09038F0
:102D500081F402C0943069F090E0009741F0EFE90F
:102D6000FFE03197F1F700C000000197F6CF81E056
:102D700001C080E09091700192FF02C091E089272C
:102D8000882311F0289A0895289808951F920F9289
:102D90000FB60F9211242F933F934F935F936F932E
:102DA0007F938F939F93AF93BF93EF93FF93809104
:102DB0000A03811122C28BB190911A03907E8F7108
:102DC000892B8BB98BB1837E90911903892B8BB999
:102DD0008091180386BD82E085BD81E080930A035F
:102DE000789480912C0390912D03892B09F0BFC01A
:102DF0008091510690917C06981709F4A4C0E09147
:102E000051062E2F30E087E0E89FF0011124EE5AA2
:102E1000F94FF0932D03E0932C03828193819093DB
:102E2000890080938800808191819093280380930A
:102E30002703E481809129038E1761F1E093290330
:102E400082E1E89FF0011124E358F94FF0932B033E
:102E5000E0932A0384859585A685B785B695A795C1
:102E6000979587958093130390931403A09315036C
:102E7000B093160380930F0390931003A093110354
:102E8000B093120380930B0390930C03A0930D0354
:102E9000B0930E03A0912A03B0912B0350969C91FE
:102EA000509780910903892780931A0387E0829FB6
:102EB000F001839FF00D1124EE5AF94F25814D91B9
:102EC0005D916D917C911397022E04C07695679564
:102ED000579547950A94D2F740931B0350931C03D0
:102EE00060931D0370931E0314964D915D916D9137
:102EF0007C911797022E04C0769567955795479554
:102F00000A94D2F740931F03509320036093210348
:102F10007093220318968D919D910D90BC91A02DD8
:102F200004C0B695A795979587952A95D2F7809373
:102F3000230390932403A0932503B0932603868153
:102F40000E94511614C00E949016E0912A03F0913D
:102F50002B038189882339F01092B3008091B0004F
:102F60008F778093B00084E00E942D1D46C1809130
:102F700019018130B1F486B18072909100018917F6
:102F800081F0109219018CE0E1E0F1E0ADE0B1E0F8
:102F900001900D928A95E1F78091070780648093F4
:102FA00007071092190340910B0350910C03609195
:102FB0000D0370910E0380911B0390911C03A0914F
:102FC0001D03B0911E03840F951FA61FB71F80938A
:102FD0000B0390930C03A0930D03B0930E03E091A9
:102FE0002A03F0912B03448555856685778548171C
:102FF00059076A077B0768F524E020931903448585
:10300000558566857785841B950BA60BB70B80933A
:103010000B0390930C03A0930D03B0930E03208930
:103020008091010190910201A0910301B0910401EE
:1030300025FF04C00197A109B10903C00196A11D94
:10304000B11D8093010190930201A0930301B093FD
:10305000040140910F03509110036091110370918E
:10306000120380911F0390912003A0912103B0913E
:103070002203840F951FA61FB71F80930F03909301
:103080001003A0931103B093120344855585668500
:103090007785481759076A077B0778F52091190348
:1030A0002860209319034485558566857785841BA0
:1030B000950BA60BB70B80930F0390931003A0936F
:1030C0001103B093120320898091050190910601AC
:1030D000A0910701B091080126FF04C00197A10942
:1030E000B10903C00196A11DB11D80930501909304
:1030F0000601A0930701B09308014091130350917A
:10310000140360911503709116038091230390912D
:103110002403A0912503B0912603840F951FA61FB9
:10312000B71F8093130390931403A0931503B093D8
:1031300016034485558566857785481759076A07BC
:103140007B0778F5209119032061209319034485AA
:10315000558566857785841B950BA60BB70B8093E9
:10316000130390931403A0931503B09316032089BF
:103170008091090190910A01A0910B01B0910C017D
:1031800027FF04C00197A109B10903C00196A11D41
:10319000B11D8093090190930A01A0930B01B09394
:1031A0000C0180911A01843039F4909119038091B7
:1031B000200189238093190380912703909128038C
:1031C00001979093280380932703892B69F4109229
:1031D0002D0310922C03809151068F5F809351062E
:1031E000863011F4109251069091190380910803D2
:1031F00089278093190310920A03FF91EF91BF91E1
:10320000AF919F918F917F916F915F914F913F917E
:103210002F910F900FBE0F901F9018958091700105
:1032200082FF02C0289A01C02898809108038093E9
:10323000190380915B01880F845081958093180356
:1032400080916F00826080936F0008954F925F922B
:103250006F927F928F929F92AF92BF92CF92DF92A6
:10326000EF92FF926B017C0180906C0190906D0158
:10327000A0906E01B0906F0140906801509069017C
:1032800060906A0170906B01A3019201C501B401C5
:103290000E94B83887FF19C06091230170E080E078
:1032A00090E00E944A372AE037ED43E25CE30E9457
:1032B000F838A70196010E94F8386B017C01A30140
:1032C00092010E94B83887FD0AC0409227015092AF
:1032D00028016092290170922A018FEF47C0A50151
:1032E0009401C701B6010E9496361816E4F020E05A
:1032F00030E0A901C701B6010E949636811109C0CC
:1033000010922701109228011092290110922A018F
:103310002DC08092270190922801A0922901B0929D
:103320002A0181E023C0C0922701D0922801E092B7
:103330002901F0922A01A5019401C701B6010E945A
:10334000A03520910403309105034091060350916C
:1033500007030E94F8380E94853720E030E040E8FB
:103360005FE30E94A1350E941937862FFF90EF90EE
:10337000DF90CF90BF90AF909F908F907F906F9095
:103380005F904F90089590911B01911126C081117B
:103390000EC010922701109228011092290110925C
:1033A0002A018091B0008F778093B00014C08031E3
:1033B00011F42D9801C02D9A9091700191FF05C0D4
:1033C000803219F440E050E0BA01CB01BA010E940A
:1033D00026190E945116109225010895CF93DF936C
:1033E000239AC0EBD0E083E0888384E08093B1002F
:1033F000259A20916C0130916D0140916E015091A0
:103400006F01609168017091690180916A019091EA
:103410006B010E94A0359B01AC0160E070E08EE77B
:1034200093E40E94A0366093040370930503809395
:1034300006039093070388818F778883DF91CF916C
:1034400008956AE080E090E00E94870245E550E040
:103450006BE271E081E090E00C94A9020F931F935E
:10346000CF93C82F8B010E9466272DE0C29FC00119
:1034700011244CE050E0B8019E5FCF911F910F9155
:103480000C94A9021F93CF93DF93182FEB018DE0CB
:10349000189FB00111247E5F4CE050E0CE010E94E5
:1034A0004302892B59F48CE0FE0111928A95E9F7C9
:1034B000BE01812F0E942E1A80E001C081E0DF91C1
:1034C000CF911F910895EF92FF920F931F93CF9387
:1034D000DF93CDB7DEB72C970FB6F894DEBF0FBEE3
:1034E000CDBF182F80FF0BC085E5ECE1F3E0ABE228
:1034F000B1E005900D928A95E1F70E94211A11FF23
:1035000010C0CE0101967C018CE0F70111928A95E2
:10351000E9F700E0B701802F0E942E1A0F5F0830F4
:10352000C9F712FF14C060E080E093E00E948702B8
:1035300060E081E093E00E94870260E081E593E033
:103540000E94870260E082E593E00E94870213FFF9
:103550000AC060E08EEA93E00E94870260E08FEA92
:1035600093E00E9487022C960FB6F894DEBF0FBE40
:10357000CDBFDF91CF911F910F91FF90EF900895F4
:103580001F920F920FB60F9211242F933F934F93D8
:103590005F936F937F938F939F93AF93BF93EF93BB
:1035A000FF93E091C600E13271F028F4E83179F43C
:1035B0000E94042956C0EF3321F0EE3741F482E037
:1035C00003C081E001C088E00E942D1D4AC0E7FFD2
:1035D00037C08E2F90E0FC01E458F109ED31F10580
:1035E00008F03FC0E659FF4F0C94433A80E2ECCF1D
:1035F00080911A0185FF35C080E4E6CF81E00DC0DF
:1036000082E00BC084E009C088E007C080E105C00B
:1036100080E203C080E401C080E80E94141D21C044
:1036200081E00BC082E009C084E007C088E005C0EB
:1036300080E103C080E201C080E40E940B1D11C044
:10364000A091980281E08A0F813809F480E090917E
:103650009702891731F0B0E0AA5EBD4FEC938093DA
:103660009802FF91EF91BF91AF919F918F917F91C0
:103670006F915F914F913F912F910F900FBE0F90DF
:103680001F9018951F920F920FB60F9211248F93CF
:103690009F93EF93FF9380910303E82FF0E0E656AA
:1036A000FD4F90819093C6008F5F893609F480E0CA
:1036B0008093030390919902891305C08091C10002
:1036C0008F7D8093C100FF91EF919F918F910F901B
:1036D0000FBE0F901F901895E091990291E09E0FF8
:1036E000993631F490E004C02091070724FD0FC003
:1036F000209103032917C1F3F0E0E656FD4F8083C4
:10370000909399028091C10080628093C1000895D6
:10371000CF93C82F85E193E00E94C3268C2F0E948F
:103720009D26CF910C94B610EF92FF920F931F93AA
:10373000CF93DF9360915B0170E080E00E94DA102C
:1037400060915E0170E081E00E94DA1060915C019E
:1037500070E082E00E94DA1060915D0170E083E029
:103760000E94DA106091700162FB662760F970E0D8
:1037700084E00E94DA106091700166FB662760F9B0
:1037800070E085E00E94DA1080917001082E000C34
:10379000990B692F661F6627661F70E086E00E94FE
:1037A000DA1060915F0170E08AE00E94DA104091C7
:1037B000600150916101609162017091630123E0A9
:1037C0008BE00E94BA1040916401509165016091B4
:1037D00066017091670123E08CE00E94BA1060914D
:1037E0007001617070E08DE00E94DA1060917001EC
:1037F00065FB662760F970E084E10E94DA10609151
:10380000700163FB662760F970E085E10E94DA10C1
:10381000609170016295617070E086E10E94DA103B
:103820006091710170E087E10E94DA1040917201AD
:1038300050917301609174017091750123E088E1EA
:103840000E94BA1040917601509177016091780101
:103850007091790123E089E10E94BA1060917A01A8
:1038600070917B018AE10E94DA1040917C015091B5
:103870007D0160917E0170917F0123E08BE10E94C8
:10388000BA10409168015091690160916A0170918C
:103890006B0120E08EE10E94BA1040916C015091C2
:1038A0006D0160916E0170916F0120E08FE10E94C7
:1038B000BA10609170016695617070E080E20E94BC
:1038C000DA10D4E6F12C0BE211E083E0E82EED0EE5
:1038D000CD2F82E0F81691F0E3E0FE16E9F0F1E07A
:1038E000FF1631F0F80140815181628173811AC065
:1038F000F801448555856685778514C020E030E061
:1039000041E655E4F801608D718D828D938D0E94A2
:10391000A036AB01BC0106C0F80144A155A166A1C7
:1039200077A1705823E08C2F0E94BA100C5F1F4FB4
:10393000CF5FEC12CECFD65FF394DC3821F6DF9167
:10394000CF911F910F91FF90EF900895811104C0C6
:1039500081E793E00C94C3260C94881BCF93DF93EC
:10396000C1E1D7E08991882319F00E946C1BFACF3E
:10397000DF91CF910895CF93DF9321E5829FC0011E
:103980001124EC01DD5F40E550E0BE0181E197E0EC
:103990000E944302892B69F4109211070E94662746
:1039A00040E550E061E177E0CE010E94A90280E0AD
:1039B00001C081E0DF91CF910895CF93DF93C0E004
:1039C0008C2F0E94BB1C81110EC0109211078EE338
:1039D0000E946C1B0E94AE1C8AE30E946C1B87E055
:1039E0000E94881B12C080911107882371F00E94E9
:1039F000F202D82F8EE30E946C1B0E94AE1C8AE359
:103A00000E946C1B8D2F0E94A61CCF5FC230C1F696
:103A1000DF91CF9108959FB7F89420910A07822BE8
:103A200080930A079FBF08959FB7F89420910907D4
:103A3000822B809309079FBF08959FB7F8948093C6
:103A400008079FBF08952FB7F894909107078095B6
:103A50008923809307072FBF08959FB7F89420917B
:103A60000707822B809307079FBF08958F929F922D
:103A7000AF92BF92CF92DF92EF92FF920F931F937C
:103A8000CF93DF93EB012BE2E22E21E0F22E8C01AB
:103A90006B018CE0C80ED11C699179918991999143
:103AA000F70181909190A190B1907F010E944A37D7
:103AB000A50194010E94A036F8016193719381934E
:103AC00091938F01CC15DD0539F7DF91CF911F91CF
:103AD0000F91FF90EF90DF90CF90BF90AF909F90AD
:103AE0008F90089596B1892F877049F0892F80951E
:103AF000817091FF826092FD03C08460089580E030
:103B000008951F920F920FB60F9211242F933F9397
:103B10004F935F936F937F938F939F93AF93BF93D5
:103B2000CF93EF93FF930E94721DC82F882389F0D3
:103B300080FD0E940429C2FF05C0809107078260B2
:103B400080930707C1FF05C08091070788608093B5
:103B50000707FF91EF91CF91BF91AF919F918F9107
:103B60007F916F915F914F913F912F910F900FBE79
:103B70000F901F9018952F923F924F925F926F92E5
:103B80007F928F929F92AF92BF92CF92DF92EF92ED
:103B9000FF920F931F93CF93DF93CDB7DEB7EC97D0
:103BA0000FB6F894DEBF0FBECDBF80911E0180FD21
:103BB00087C79091510680910B07981709F480C729
:103BC00080910E0790910F07892B09F015C3109172
:103BD0001E0112FF09C08091500622E3289FC001F8
:103BE0001124805D9C4F02C00E94562790930F07BE
:103BF00080930E0720900E0730900F072114310498
:103C000009F45EC70091D806802F817000FF03C0C1
:103C10001092D806EAC09091D7069F5F953009F0C0
:103C2000892F8093D706E82EF12C32E13E9DF001DA
:103C30003F9DF00D1124E358F94FF0930D07E093E9
:103C40000C07D10150969C915097908BE2E18E9F8A
:103C5000C001112420E030E04D915D916D917D9186
:103C6000F901E80FF91FE358F94F689412F8440F6F
:103C7000551F661F771F1694D1F7408351836283C7
:103C800073832C5F3F4F2C30310531F722E12E9D9D
:103C9000F0012F9DF00D11249F012358394FF101A0
:103CA00084859585A685B78543E0880F991FAA1F4F
:103CB000BB1F4A95D1F7F90184879587A687B787F7
:103CC000D1011C966D917D918D919C911F970E94C1
:103CD00048376093DD067093DE068093DF0690938D
:103CE000E006F101268D378D40A151A10E94A0363A
:103CF0009B01AC016093E1067093E2068093E306BA
:103D00009093E40660E070E080EA9FE30E94A036B2
:103D10006093E5067093E6068093E7069093E806C5
:103D20001092D9061092DA061092DB061092DC0689
:103D300011FD02C003FF1FC06091F6067091F706E7
:103D40008091F8069091F9066093EE067093EF0665
:103D50008093F0069093F1069B01AC010E94F83825
:103D6000D10152966D937D938D939C935597077FC8
:103D70000093D8060FC0F1016289738984899589FF
:103D80000E9497396093EE067093EF068093F006D9
:103D90009093F106F2E1FE9DC001FF9D900D11246C
:103DA0009C012358394F7901D90151961C92809179
:103DB000700181FF1AC0F101818985FF16C022A51B
:103DC00033A544A555A560E070E080E89FE30E941C
:103DD000A0366093020770930307809304079093C3
:103DE0000507E1E0D7015196EC931092EA06109294
:103DF000EB061092EC061092ED06D1015A962D9129
:103E00003D914D915C915D9729833A834B835C830F
:103E100060E070E080E09FE30E94A0364B015C010F
:103E2000F101468C578C60A071A011FF4BC0F2E0ED
:103E3000F093E906D1015296CD90DD90ED90FC9083
:103E40005597A70196010E94F8389B01AC01C30168
:103E5000B2010E94A0354B015C0120E030E0A901D5
:103E60000E94963687FF1DC029813A814B815C8173
:103E7000CA01B9010E94A135A30192010E94F8383C
